:020000040000fa
:0800000082050400000000006d
:020000040000fa
:020000040002f8
:04afe000dfff00008f
:020000040000fa
:020000040002f8
:04afe400ffff00006b
:020000040000fa
:020000040002f8
:04afe80078ff0000ee
:020000040000fa
:020000040002f8
:04afec007dff0000e5
:020000040000fa
:020000040002f8
:04aff00078ff0000e6
:020000040000fa
:1000080000000000000000000000000000000000e8
:100018007a05000000000000000000000000000059
:10002800cc0900000000000000000000580a000091
:1000380000000000000000000000000000000000b8
:10004800880a00000000000000000000580b0000b3
:10005800c40b0000f40b00000000000000000000ca
:100068000000000000000000000000000000000088
:100078000000000000000000000000000000000078
:10008800000000000000000000000000b40a0000aa
:10009800280b000000000000000000000000000025
:1000a8000000000000000000000000000000000048
:1000b8000000000000000000000000000000000038
:1000c8000000000000000000000000000000000028
:1000d8000000000000000000000000000000000018
:1000e8000000000000000000000000000000000008
:1000f80000000000000000000000000000000000f8
:1001080000000000000000000000000000000000e7
:1001180000000000000000000000000000000000d7
:1001280000000000900b000000000000000000002c
:1001380000000000000000000000000000000000b7
:1001480000000000000000000000000000000000a7
:100158000000000000000000000000000000000097
:100168000000000000000000000000000000000087
:100178000000000000000000000000000000000077
:100188000000000000000000000000000000000067
:1001980000000000000000005c0c0000880c00005b
:1001a800b40c000000000000000000000000000087
:1001b8000000000000000000000000000000000037
:1001c8000000000000000000000000000000000027
:1001d8000000000000000000000000000000000017
:1001e8000000000000000000000000000000000007
:1001f80000000000000000000000000000000000f7
:1002080000000000000000000000000000000000e6
:1002180000000000000000000000000000000000d6
:1002280000000000000000000000000000000000c6
:1002380000000000000000000000000000000000b6
:1002480000000000000000000000000000000000a6
:100258000000000000000000000000000000000096
:100268000000000000000000000000000000000086
:0c0278000000000000000000000000007a
:020000040000fa
:10040000803e2000030007008100e900fcff3a0065
:1004100000000600831f7800c20320000400bc0017
:1004200066015100e0815900f23fb1000380b10044
:1004300006003500ee03090000000000423fb10055
:100440000380b100fbff3d001200b000223fb0006e
:10045000020035000280090000000000cf01780092
:1004600000000600861f78006022b8000602200007
:100470000000d0008180d2000482d2008582d200a8
:100480000000a0000202520083825a0003003100e3
:100490000202420083824a000000a1000603e90034
:1004a000f3ff3a004f03780000000600889fbe006b
:1004b0008a9fbe008c1f78000004be004101070027
:1004c0000478a30026003a006120e10025003200f4
:1004d00009f8a30025003a006420e1002100320061
:1004e000f507b1000508a30002003200000040003b
:1004f000818048006044b800031020000200200002
:1005000000004000818048000805440089854c00b7
:100510000a0541008b8549000a0550008b8558006b
:10052000030033000a00be000204740083847400d8
:100530008301d1000281d300830f7100f0ff3a00e4
:100540008904d1000884d300600149008201780049
:10055000c1adde00fb07b0002f0107000700370028
:100560000960a0000800be0004003700120220004d
:1005700062928800f0ff2f00f1ff27004f067800fd
:100580004f05be004f04be000000060003f0a200ad
:10059000869fbe00889fbe008a9fbe008c9fbe00c3
:1005a00000010700420133006450e1004f003200b7
:1005b0006420e1005200320003826c0007003b001f
:1005c0000905d0000306d000820f54000c065d0020
:1005d0000200390002003200890178000306780029
:1005e0008582550004003d000003fd008103fd00ed
:1005f0008502ea008b854200840f720002003b00f6
:1006000060001000e08018006011b8000005eb00e9
:100610007a28e1000a00390006007800c75ddd0095
:10062000f707b200878075002d00370082817100c6
:100630000a017800610560008180d1000080d3004c
:100640008502e900f9ff3b0006044000878448006a
:1006500002003b0060041400e0841c000988a30031
:10066000070032008a81710082817100610164009b
:100670008904d1000884d3008b05e80017003700f7
:100680000978a30013003a000b00e00013003400c7
:100690008b05e9000804440089844c000a44740076
:1006a0000978a3000d003a000b00e00007003400b9
:1006b0008b05e9000804440089844c0001003a00dd
:1006c0000b0020000978a300f7ff32000001eb00c7
:1006d00002003700828171000a017800ce00070015
:1006e0000cf0a70001f0a000fa0037006420e10040
:1006f00002003a00838f6c00fb0033000801be004b
:100700000200be00f3003700869fbe00889fbe0037
:100710008a9fbe008c9fbe00a2000700e400330049
:1007200003866c006450e100240032006420e10084
:10073000270032006150e100220032006120e10018
:10074000210032008b854200eb07b1000134b80074
:10075000003ab8000804420089844a00013ab8000f
:100760000030b8008880400009014a0004003300ce
:100770000000400081804800020149008b05e9002b
:10078000c909dd0083017000010032001300200060
:10079000c814de004814dd004709de001200b20074
:1007a000c808de00088470009b00070001f0a1006b
:1007b0000cf0a70001f0a000c60037006120e100a6
:1007c000c90032000801be000200be00f7ff37007a
:1007d0006150e100fcff3a00c3003700829fbe0079
:1007e0000001be00770007000470a70003f0a1001d
:1007f0006509b100180032000e0035006828e100dc
:1008000007003500f0ff2f00f1ff27000300e00094
:1008100015003b00010028004f01be00000005004c
:1008200000004000818048008502e900fcff3a009a
:1008300009003700f88f420003003c008000eb0005
:100840004f01be00000005008100d1000080d300f0
:100850008502e800fcff3a000300e00002003b00d4
:1008600060001000e08018004f01be00000006008c
:10087000829fbe000001be00520007000470a70066
:1008800003f0a10003f8a30015003a006509b100c8
:10089000110032000a0035006928e100030035002c
:1008a000010028004f01be000000050000004000cc
:1008b000818048008502e900fcff3a00060037000d
:1008c000f88f4200060035008100d1000080d3007f
:1008d0008502e800fcff3a004f01be000000060060
:1008e0008000eb004f01be00000005008000eb001f
:1008f000829fbe00889fbe008a9fbe0001057800cf
:100900000100e0000400350008003c000000e000a9
:10091000200032000500370060001000e080180061
:1009200002003b0001f024001a0037000004be0062
:100930006011b8006b0920000982cf000200390065
:100940000882cf000441b000694252000e0032001c
:1009500008003b0082817100610164008904d100bc
:100960000884d3008b05e8000442e800f9ff3a0050
:10097000050037000804440089844c008b05e90019
:100980000442e900fbff3a00230007000af0a70039
:1009900001f0a0004f05be004f04be004f01be0095
:1009a000000006000004be00060007000003be00b1
:1009b0000405be000200be0002000700844f75005f
:1009c00000000600c70ade00f107b200f50fb20012
:1009d00008003200e1cf4200020032000170a000a6
:1009e00024000500810f700001003200040805009a
:1009f00044000500810f700002003a001400050059
:100a00008502e9000000400081c04800fcff3b0077
:100a10000170a000240005008100200061805500c5
:100a20000b003d000b00200061fe2f000100e100e3
:100a30001d00340082817100610164008904d100cd
:100a40000884d3000000e800faff3a00710020009b
:100a500061006400030070000200600009003200c1
:100a600061044400e0844c000988a50005003200c0
:100a70008b05e8006808e10002003a008904d10013
:100a80000884d300f20f20000258e10005003d0069
:100a9000c75ddd00f907b2008980750008007800a5
:100aa000000006000bf827008b007800000005000e
:100ab0000200be006450e100050036006420e10041
:100ac000020036000968a30001003a000800be00d9
:100ad0000160a0004f06be004f05be004f04be00df
:100ae0004f03be0000000600f0ff2f00f1ff2700bb
:100af000f8ff37000020ef000220ef00c088a900b7
:100b0000004006000f002100403221000001880053
:100b1000000000000000eb00000778000c00090056
:100b2000002f78000007eb005420ef000e2eef009e
:100b30001e2eef000000eb0001242100bf1d090064
:100b40008018780040a7a900a10020002cfe070013
:100b5000e0022000303a880044e7a90044c7a90019
:100b60004407a9004427a9004447a9004467a900f5
:100b70004487a900300020000600fc0031742000ea
:100b800082072000a309200082487800834878006b
:100b900080487800113a8000618070000600fc00f7
:100ba0002174200062042000730520008248780030
:100bb00083487800804878004427ef00e002200056
:100bc000303a8800300020000d00fc003174200015
:100bd00082072000a309200082487800834878001b
:100be000804878000000200021742000620420006a
:100bf0007305200082487800834878008048780098
:100c000042a7ae00feff3700813e2000fcfd07003a
:100c100010c0b30086e6b70090c2b300c4e6b700c8
:100c2000000ea800007825008070880010cea90072
:100c3000108ea90010aea900008ea9004188a8005e
:100c400041a8a90041c8a90004a1a8000481a800e6
:100c500005e1a8000068a9000021ef0002a1ef0053
:100c60002068a8001061a8001021a90011e1a800c7
:100c700011a1a90010a1a8001081a8000621ef0071
:100c80000a21ef000ca1ef000ea1ef004408a9001b
:100c90004428a9004448a9000108a9002108a80087
:100ca0001fe1a8001fa1a9001ec1a9001ea1a80044
:100cb0001e81a8001e61a9001e21a9004d88a80060
:100cc0004da8a8004dc8a900803e2000d00888008b
:100cd0000368a9002368a80021e1a80021a1a900b8
:100ce00020c1a90020a1a8002081a8002021a900de
:100cf0004e08a8004e28a9004e48a8000388a90065
:100d0000a00e2000e00888002388a8002002a90087
:100d10002022a9002042a90020a2a9002062a90047
:100d20002082a90020e2a9002102a9002122a90015
:100d3000700720004011880022a2a90022c2a90049
:100d400022e2a90021e2a8002182a9004588a90089
:100d500045a8a80045c8a8002168a8002828a80020
:100d600023e2a9002342a8002362a9000188a90068
:100d70002188a8004608a9004628a8004648a800df
:100d80000e0ea80021e3a9002143a80021a3a90079
:100d90002123a9002103a90020e3a90020c3a90061
:100da00020a3a9002083a9002043a80023e3a900d1
:100db00023c3a90023a3a9002343a9002323a90037
:100dc0002303a90022c3a90022a3a9002283a9000a
:100dd0002263a9002243a9002223a9002203a9001b
:100de0002563ef0024e3ef003223ef002823ef0018
:100df0002623ef002e23ef003023ef0021a8a800c8
:100e000046c8a80046a8a9004688a80001a8a900cd
:100e100021e3a8004008a9004028a9004048a800f4
:100e20002008a8000008a900c208a80080c0b300dc
:100e3000c8e8b7002bc8a9002be8a9002c08a90016
:100e40000bc8a9000be8a9000c08a90001eca90037
:100e500001aca900016ca900014ca900012ca9005a
:100e6000010ca90000eca900008ca90000aca900ad
:100e700000cca900000ca900002ca900004ca9007e
:100e8000006ca900202cef00402cef00602cef003c
:100e90000000210020608800020ca900022ca9009b
:100ea000024ca900262cef00462cef00662cef0028
:100eb000282cef00482cef00682cef000aacef0064
:100ec00023eca80023cca80023aca900238ca90004
:100ed000236ca900234ca800232ca900230ca900f3
:100ee000222ca80043eca80043cca80043aca900e6
:100ef000438ca900436ca800434ca900432ca900d3
:100f0000430ca90063eca80063cca80063aca90063
:100f1000638ca800636ca800634ca900dabc2a00ab
:100f20001b32240030002c00fa608800fb6088002f
:100f300020618800dabc2a001b32240020402c00eb
:100f4000fa608800fb60880010618800dabc2a0023
:100f50001b32240030002c00fa608800fb608800ff
:100f600020628800dabc2a001b32240000802c009a
:100f7000fa608800fb60880010628800dabc2a00f2
:100f80001b32240030002c00fa608800fb608800cf
:100f900020638800dabc2a001b32240000802c0069
:100fa000fa608800fb60880010638800a7003700a3
:100fb0003f00370000202000006188000020200052
:100fc000006288000020200000638800020ca90055
:100fd000022ca800024ca80004acef0028acef00e3
:100fe00048acef0068acef00262cef00462cef0079
:100ff000662cef000aacef0023eca80023cca9007c
:1010000043eca80043cca90063eca80063cca90082
:10101000dabc2a001b32240030002c00fa60880061
:10102000fb60880020618800dabc2a001b322400a3
:1010300000002800fa608800fb60880010618800ca
:10104000dabc2a001b32240030002c00fa60880031
:10105000fb60880020628800dabc2a001b32240072
:1010600000002800fa608800fb6088001062880099
:10107000dabc2a001b32240030002c00fa60880001
:10108000fb60880020638800dabc2a001b32240041
:1010900000002800fa608800fb6088001063880068
:1010a00011eea90011aea900116ea900670037006a
:1010b000350037000010200000618800001020007b
:1010c000006288000010200000638800020ca90064
:1010d000022ca800024ca8000a2cef0004acef0080
:1010e000282cef005055250040628800a0aa2a0055
:1010f00040638800dabc2a001b32240030002c0038
:10110000fa608800fb60880020618800dabc2a0051
:101110001b32240000002c00fa608800fb6088006d
:1011200010618800dabc2a001b32240030002c0039
:10113000fa608800fb60880020628800dabc2a0020
:101140001b32240000002c00fa608800fb6088003d
:1011500010628800dabc2a001b32240030002c0008
:10116000fa608800fb60880020638800dabc2a00ef
:101170001b32240000002c00fa608800fb6088000d
:101180001063880031003700300037000010200065
:10119000006188000010200000628800020ca90095
:1011a000022ca800024ca8000a2cef0004acef00af
:1011b000282cef000000240040628800dabc2a00de
:1011c0001b32240030002c00fa608800fb6088008d
:1011d00020618800dabc2a001b32240000002c00a9
:1011e000fa608800fb60880010618800dabc2a0081
:1011f0001b32240030002c00fa608800fb6088005d
:1012000020628800dabc2a001b32240000002c0077
:10121000fa608800fb60880010628800dabc2a004f
:101220001b32240030002c00fa608800fb6088002c
:1012300020638800dabc2a001b32240000002c0046
:10124000fa608800fb60880010638800218ca90088
:10125000418ca900618ca900216ca900416ca900f6
:10126000616ca900214ca900414ca900614ca90066
:1012700020eca80040eca80060eca8003e2cef0099
:101280005e2cef007e2cef0001eca8007eb2ef0098
:101290000000eb00619d2100ff00090080587800ec
:1012a000a372ef00a472ef009232ef009432ef00cd
:1012b0000000eb0061ad2100ff00090080587800bc
:1012c000a572ef00a672ef000080eb00219c2100c8
:1012d00009000900801878000000eb00212c210093
:1012e000ff00090080187800b772ef00b872ef00b5
:1012f0000000eb00214c2100ff000900801878005d
:10130000b972ef00108ea900148ea900008ea900fa
:10131000048ea90010aea90014aea9002008a800f0
:101320002068a80021a8a80001a8a900262cef0089
:101330002003a9002023a80000122000e008880054
:101340000388a9002388a800803e2000d0088800d8
:101350000368a9002368a80000802000709388001b
:101360007c32ef007a32ef007832ef0000c4b30035
:1013700080f2b70000c4b30082f2b700a0c0b3008f
:1013800086f2b700400020004094880096060700cf
:101390009507070097013700ff3ffc004200f80067
:1013a0003600f8004400f8008e1f78000e00200080
:1013b0000d000900be1f78003200f8004012f8004e
:1013c0004212f8000100fc000008a9006412ae00ff
:1013d0000c0037000021ef006412a9006832ef0012
:1013e000ba72ec00bad2bf000080fb000000d0004f
:1013f000216c21000100400001002000010878005c
:101400001e00370000088000309388004093800061
:1014100001002000f21f2000030020000001410015
:10142000818149003093800001002000820f50002c
:10143000838f58000f0036000021ef006832ef0064
:10144000ba72ec00329380000300200000002000fc
:101450001100200003fc0700a12b2100914078001f
:101460008180fb0081804000226c21008030790067
:10147000020037003093800040938800ff3ffc005b
:101480004212f9004012f9003200f900ae012000ca
:101490000d0009004f1778004f0778004400f9004d
:1014a0003600f9004200f9000100fc00004006008f
:1014b000ff3ffc004200f8003600f8004400f8004e
:1014c0008e1f78000e0020000d000900be1f78005e
:1014d0003200f8000100fc000068a9000021ef00c4
:1014e0006412a800ff3ffc003200f900ae012000aa
:1014f0000d0009004f1778004f0778004400f900ed
:101500003600f9004200f9000100fc00004006002e
:10151000ff3ffc004200f8003600f8004400f800ed
:101520008e1f78000e0020000d000900be1f7800fd
:101530003200f8000100fc000108a900ff3ffc0098
:101540003200f900ae0120000d0009004f177800ad
:101550004f0778004400f9003600f9004200f90016
:101560000100fc0000400600ff3ffc004200f800c4
:101570003600f8004400f8008e1f78000e002000ae
:101580000d000900be1f78003200f8004012f8007c
:101590000100fc000368a9001421ef006a32ef008b
:1015a0005032ef00bad2bf00bb52e3000a00320053
:1015b000bb72ec005032ec00bbd2bf000080fb00dd
:1015c00000004000216c2100608078006a12b400a5
:1015d00050938800f3ff37005012e20007003600f6
:1015e00050938000829280000200e00002003200ee
:1015f000110009000280d80050938800800c200060
:101600000100200092948000a39480000201400019
:101610008381480092ce8800a3ce8800b612a8002d
:10162000ff3ffc004012f9003200f900ae0120003b
:101630000d0009004f1778004f0778004400f900ab
:101640003600f9004200f9000100fc0000400600ed
:10165000ff3ffc004200f8003600f8004400f800ac
:101660008e1f78000e0020000d000900be1f7800bc
:101670003200f8000100fc000388a9001821ef00e7
:101680002023a900ff3ffc003200f900ae0120003a
:101690000d0009004f1778004f0778004400f9004b
:1016a0003600f9004200f9000100fc00004006008d
:1016b000ff3ffc004200f8003600f8004400f8004c
:1016c0008e1f78000e0020000d000900be1f78005c
:1016d0003200f8000100fc000168a900a372ec00d0
:1016e000a3d2bf008080fb0030118000629d2100ea
:1016f00080707900ff3ffc003200f900ae0120004d
:101700000d0009004f1778004f0778004400f900da
:101710003600f9004200f9000100fc00004006001c
:10172000ff3ffc004200f8003600f8004400f800db
:101730008e1f78000e0020000d000900be1f7800eb
:101740003200f8000100fc000828a9002242ae0087
:10175000000037002222af002222a900ff3ffc0038
:101760003200f900ae0120000d0009004f1778008b
:101770004f0778004400f9003600f9004200f900f4
:101780000100fc0000400600ff3ffc004200f800a2
:101790003600f8004400f8008e1f78000e0020008c
:1017a0000d000900be1f78003200f8000100fc00a7
:1017b0000188a900128eaa00108ea900ff3ffc002c
:1017c0003200f900ae0120000d0009004f1778002b
:1017d0004f0778004400f9003600f9004200f90094
:1017e0000100fc0000400600ff3ffc004200f80042
:1017f0003600f8004400f8008e1f78000e0020002c
:101800000d000900be1f78003200f8000100fc0046
:1018100001a8a9002003a900001880006093880097
:101820007093800061938000808f50000400360028
:10183000709380006c12b500b093880003003700ed
:10184000609380006e12b500b0938800a093800072
:101850007612b40090938800b0938000a093880023
:1018600060938000709388008007200001002000b2
:1018700092948000a394800002014000838148007c
:1018800072ce880083ce8800b612a800ff3ffc000d
:101890003200f900ae0120000d0009004f1778005a
:1018a0004f0778004400f9003600f9004200f900c3
:1018b0000100fc0000400600ff3ffc004200f80071
:1018c0003600f8004400f8008e1f78000e0020005b
:1018d0000d000900be1f78003200f8000100fc0076
:1018e0000bc8a900ff3ffc003200f900ae01200048
:1018f0000d0009004f1778004f0778004400f900e9
:101900003600f9004200f9000100fc00004006002a
:10191000ff3ffc004200f8003600f8004400f800e9
:101920008e1f78000e0020000d000900be1f7800f9
:101930003200f8000100fc000be8a900ff3ffc00aa
:101940003200f900ae0120000d0009004f177800a9
:101950004f0778004400f9003600f9004200f90012
:101960000100fc0000400600ff3ffc004200f800c0
:101970003600f8004400f8008e1f78000e002000aa
:101980000d000900be1f78003200f8000100fc00c5
:101990000c08a900ff3ffc003200f900ae01200056
:1019a0000d0009004f1778004f0778004400f90038
:1019b0003600f9004200f9000100fc00004006007a
:1019c000a4d2bf00a352e30007003200a472ec00cf
:1019d000a4d2bf000080fb00619d210060c07800a0
:1019e000a7f2b70001003700a7f2ef0000000600e1
:1019f00000000600f1938000e18f50000d003a00d6
:101a000050088000a09488003008800090948800de
:101a100010d825005100200092948000a3948000eb
:101a2000020140008381480052ce880063ce8800c6
:101a30007e32ef0050088000a094880030088000bb
:101a400090948800deff070080ceb300a752b50057
:101a500006003900e0cfb300a752b50001003900fd
:101a600001003700a872ef007b013700a7f2ae003b
:101a700037003700a872ef0070c8b300a752e30028
:101a800005003a00a7d2bf00a8f2b700a9f2ef0004
:101a9000aaf2ef002d00370070c9b300a752e3008f
:101aa00005003a00a7d2bf00a8f2b700abf2ef00e2
:101ab000acf2ef002500370070cab300a752e30074
:101ac00005003a00a7d2bf00a8f2b700adf2ef00c0
:101ad000aef2ef001d00370070cbb300a752e30059
:101ae00005003a00a7d2bf00a8f2b700aff2ef009e
:101af000b0f2ef001500370070ccb300a752e3003e
:101b000004003a00a7d2bf00a8f2b700b1f2ef007c
:101b10000e00370070cdb300a752e30004003a0076
:101b2000a7d2bf00a8f2b700b2f2ef00070037005b
:101b300070ceb300a752e30004003a00a7d2bf0062
:101b4000a8f2b700b3f2ef00b4f2ef0042013700a1
:101b5000a852e20002003a003f0137003e01370080
:101b600070c8b300a852e3003d003a0000e0ef0067
:101b7000a952e30003003a00a7d2bf00a9f2b700c0
:101b800036003700a7d2bf00aaf2b700a9d2bf0023
:101b9000f1c2b30080cf100016003600e0c4b300dd
:101ba000a952e30013003e00a572ec00a5d2bf00cd
:101bb0000080fb007208200061ad210002f0780077
:101bc000a572ec00a5d2bf000081fb0061ad210031
:101bd000a9d2bf0000f17800a572ec00a5d2bf0029
:101be0000081fb0061ad2100aad2bf0000f17800a6
:101bf00019003700a9d2bf00f1c6b30080cf100092
:101c000015003600f0c7b300a952e30012003e00f1
:101c1000a572ec00a5d2bf000080fb007208200076
:101c200061ad210002f07800a572ec00a5d2bf00e2
:101c30000081fb0061ad2100a9d2bf0000f1780056
:101c4000a572ec00a5d2bf000081fb0061ad2100b0
:101c5000aad2bf0000f17800a9f2ef00fe00370021
:101c600070c9b300a852e30073003a0000e0ef002f
:101c7000ab52e30003003a00a7d2bf00abf2b700bb
:101c80006c003700a7d2bf00acf2b700ac52e20044
:101c900034003a00abd2bf00f1c2b30080cf1000d5
:101ca00016003600e0c4b300ab52e30013003e0060
:101cb000a572ec00a5d2bf000080fb0072092000d5
:101cc00061ad210002f07800a572ec00a5d2bf0042
:101cd0000081fb0061ad2100abd2bf0000f17800b4
:101ce000a572ec00a5d2bf000080fb00020020001e
:101cf00061ad210002f0780019003700abd2bf00bf
:101d0000f1c6b30080cf100015003600f0c7b30055
:101d1000ab52e30012003e00a572ec00a5d2bf005a
:101d20000080fb007209200061ad210002f0780004
:101d3000a572ec00a5d2bf000081fb0061ad2100bf
:101d4000abd2bf0000f17800a572ec00a5d2bf00b5
:101d50000080fb000200200061ad210002f078004d
:101d600034003700abd2bf00f1c2b30080cf100007
:101d700016003600e0c4b300ab52e30013003e008f
:101d8000a572ec00a5d2bf000080fb007209200004
:101d900061ad210002f07800a572ec00a5d2bf0071
:101da0000081fb0061ad2100abd2bf0000f17800e3
:101db000a572ec00a5d2bf000081fb0061ad21003f
:101dc000acd2bf0000f1780019003700abd2bf00e1
:101dd000f1c6b30080cf100015003600f0c7b30085
:101de000ab52e30012003e00a572ec00a5d2bf008a
:101df0000080fb007209200061ad210002f0780034
:101e0000a572ec00a5d2bf000081fb0061ad2100ee
:101e1000abd2bf0000f17800a572ec00a5d2bf00e4
:101e20000081fb0061ad2100acd2bf0000f1780061
:101e3000abf2ef008800370070cab300a852e3008d
:101e400023003a0000e0ef00ad52e30003003a0047
:101e5000a7d2bf00adf2b7001c003700a7d2bf0069
:101e6000aef2b700add2bf00f1c2b30080cf100018
:101e70001500360010c6b300ad52e30012003e005c
:101e8000a572ec00a5d2bf000080fb00720a200002
:101e900061ad210002f07800a572ec00a5d2bf0070
:101ea0000081fb0061ad2100add2bf0000f17800e0
:101eb000a572ec00a5d2bf000081fb0061ad21003e
:101ec000aed2bf0000f17800adf2ef006200370043
:101ed00070cbb300a852e3000a003a0000e0ef0024
:101ee000af52e30003003a00a7d2bf00aff2b70041
:101ef00003003700a7d2bf00b0f2b700bb02070053
:101f00005500370070ccb300a852e3002a003a0015
:101f100000e0ef00b152e30026003a00a7d2bf0074
:101f2000b1f2b700b152e2000d003a00a572ec0028
:101f3000a5d2bf000080fb00720c200061ad210023
:101f400002f07800a572ec00a5d2bf000081fb0072
:101f500061ad2100b1d2bf0000f17800150037005b
:101f6000b1d2bf00b1c0b30080cf10001000360066
:101f700070c1b300b152e3000d003e00a572ec0049
:101f8000a5d2bf000080fb00720c200061ad2100d3
:101f900002f07800a572ec00a5d2bf000081fb0022
:101fa00061ad2100b1d2bf0000f17800010037001f
:101fb0008c0207002800370070cdb300a852e30060
:101fc00007003a0000e0ef00b252e30003003a00dd
:101fd000a7d2bf00b2f2b700b2f2ef001e00370086
:101fe00070ceb300a852e3001b003a0000e0ef00ff
:101ff000b352e30003003a00a7d2bf00b3f2b70028
:1020000015003700a7d2bf00b4f2b700a572ec00ec
:10201000a5d2bf000080fb00720e200061ad210040
:1020200002f07800a572ec00a5d2bf000081fb0091
:1020300061ad2100b3d2bf0000f17800a572ec00c1
:10204000a5d2bf000081fb0061ad2100b4d2bf006a
:1020500000f17800b3f2ef007a12e20041013a0099
:1020600094d2bf008ed2b6001040b200e60032001b
:102070008e12a8009412ae008e12a900b9d2bf0031
:102080000080fb0000004000214c210060807800af
:10209000429480000200e0000200320011000900ba
:1020a0000280d8005094880051948000ee8f500038
:1020b00002003600e0002000509488005294800016
:1020c00060bd210060407900bcf2b700b7d2bf000c
:1020d0000080fb0000004000212c210060c078003f
:1020e000c0f2b70086d2bf00c052e30056003600ef
:1020f000a572ec00a5d2bf000080fb007209200091
:1021000061ad210002f07800a572ec00a5d2bf00fd
:102110000081fb0061ad2100bcd2bf0000f178005e
:10212000a572ec00a5d2bf000081fb0061ad2100cb
:10213000c0d2bf0000f17800bcd2bf00bdf2b70032
:102140008c32ae0013003700a572ec00a5d2bf00a0
:102150000080fb007208200061ad210002f07800d1
:10216000a572ec00a5d2bf000080fb009207200002
:1021700061ad210002f07800a572ec00a5d2bf008d
:102180000080fb000200200061ad210002f0780019
:102190008c32a9008c12af0013003700a572ec003e
:1021a000a5d2bf000080fb007209200061ad2100b4
:1021b00002f07800a572ec00a5d2bf000080fb0001
:1021c0000207200061ad210002f07800a572ec004a
:1021d000a5d2bf000080fb00f207200061ad210006
:1021e00002f078008c12a800c093800080948800d0
:1021f00020fe2f008094880080948000fe0f500005
:1022000002003400e0012000809488008002200059
:102210009012b400000678000c064600208c2100c5
:1022200060007e0092948000a39480000000410032
:10223000e08049000001be0012ce880023ce880055
:10224000b612a80042003700bd52e2001600360068
:10225000a572ec00a5d2bf000080fb007208200030
:1022600061ad210002f07800a572ec00a5d2bf009c
:102270000081fb0061ad2100bdd2bf0000f17800fc
:10228000a572ec00a5d2bf000080fb000200200078
:1022900061ad210002f07800bd72ef00c2b9ef001d
:1022a000c4b9ef00b612a8008c32af00130037009b
:1022b000a572ec00a5d2bf000080fb0072092000cf
:1022c00061ad210002f07800a572ec00a5d2bf003c
:1022d0000080fb009207200061ad210002f0780031
:1022e000a572ec00a5d2bf000080fb00f207200021
:1022f00061ad210002f078008c32a8008c12ae0093
:1023000013003700a572ec00a5d2bf000080fb00cf
:102310007208200061ad210002f07800a572ec0087
:10232000a5d2bf000080fb000207200061ad2100a4
:1023300002f07800a572ec00a5d2bf000080fb007f
:102340000200200061ad210002f078008c12a9008b
:102350006412ae00160037008c52af001300370035
:10236000a572ec00a5d2bf000080fb00720920001e
:1023700061ad210002f07800a572ec00a5d2bf008b
:102380000080fb002207200061ad210002f07800f0
:10239000a572ec00a5d2bf000080fb00f207200070
:1023a00061ad210002f078008c52a80015003700c2
:1023b0008c52ae0013003700a572ec00a5d2bf000e
:1023c0000080fb007208200061ad210002f078005f
:1023d000a572ec00a5d2bf000080fb002207200000
:1023e00061ad210002f07800a572ec00a5d2bf001b
:1023f0000080fb000200200061ad210002f07800a7
:102400008c52a90057003700010020009472af00e1
:102410001140b0008e32af001140b10051003200c7
:102420008e32a8009472ae008e32a900b9d2bf00dd
:102430000080fb0000004000214c210060807800fb
:1024400062002000110009000280d800509488002a
:1024500051948000f58f500002003600500120009a
:10246000509488005294800060be21006040790042
:10247000bef2b700b7d2bf000080fb0000004000f2
:10248000212c210060c07800c0f2b70086d2bf00c6
:10249000c052e3001d003600bfd2bf00be52e300b1
:1024a00019003200c072d500c072d500a572ec00d0
:1024b000a5d2bf000080fb00720a200061ad2100a0
:1024c00002f07800a572ec00a5d2bf000081fb00ed
:1024d00061ad2100bed2bf0000f17800a572ec0012
:1024e000c0d2bf000080fb00f005b000512a2100df
:1024f000914078008180fb0062ad210080707900fe
:10250000bed2bf00bff2b70016003700bf52e200d4
:102510001400360014aea900a572ec00a5d2bf00cd
:102520000080fb00720a200061ad210002f07800fb
:10253000a572ec00a5d2bf000081fb0061ad2100b7
:10254000bfd2bf0000f17800a572ec00a5d2bf0099
:102550000080fb000200200061ad210002f0780045
:10256000bf72ef00b612af000001070050c0b30009
:10257000b552b500e800310092948000a394800029
:10258000b0948000c1948000800f5100818f590069
:10259000d800390099f2a800b552e20041003a0093
:1025a000bd52e2003c003600c09380007812b400b7
:1025b0008094880020fe2f00809488008094800002
:1025c000fe0f500002003400e001200080948800db
:1025d000800220009012b400000678000c0646002d
:1025e000208c210060007e0092948000a3948000e3
:1025f00000004100e08049000001be0012ce8800ca
:1026000023ce8800a572ec00a5d2bf000080fb009d
:102610007209200061ad210002f07800a572ec0083
:10262000a5d2bf000081fb0061ad2100bdd2bf007b
:1026300000f17800a572ec00b7d2bf000080fb006b
:1026400000004000212c210060c07800512a2100a8
:10265000914078008180fb0062ad2100807079009c
:10266000800220009012b400000678000c0646009c
:10267000208c210060007e0092948000a394800052
:1026800000004100e08049000001be0012ce880039
:1026900023ce880002003700c2b9ef00c4b9ef00b2
:1026a0009300370010c0b300b552e30018003a00a1
:1026b000bf52e20013003600a572ec00a5d2bf00a5
:1026c0000080fb00720a200061ad210002f078005a
:1026d000a572ec00a5d2bf000081fb0061ad210016
:1026e000bfd2bf0000f17800a572ec00a5d2bf00f8
:1026f0000080fb000200200061ad210002f07800a4
:10270000bf72ef00c6b9ef00c8b9ef00780037001c
:1027100020c0b300b552e30004003a00b001070046
:10272000cab9ef00ccb9ef007100370030c0b30078
:10273000b552e3002a003a00f2948000039580002d
:1027400020852b00e1f72300eff707002092880097
:10275000319288009093800064f807000001be0069
:10276000a0702d0031ba2300e7f707002292800005
:102770003392800086f70700f09488000195880066
:10278000b772ec00f29480000395800000002000f6
:1027900001082400dcf7070044f7070034f80700bd
:1027a000801f7800b7d2bf000081fb00020141000a
:1027b000212c21004fb17800b7d2bf000080fb0070
:1027c00000004000212c2100608078004500dd00e1
:1027d00030638800ceb9ef00d0b9ef004400370075
:1027e00040c0b300b552e30041003a00b7d2bf0089
:1027f0000080fb0000004000212c21006080780058
:102800008000780086d2bf000080fb00810f50005e
:10281000030036006a12e200010036006a32ed0061
:10282000d2948000e39480003033230031f72300fa
:10283000b5f70700209288003192880050938000fd
:102840002af807000001be00d0cc2c00c1d4230020
:10285000adf7070022928000339280004cf707000a
:10286000d0948800e1948800b972ec00d094800084
:10287000e1948000fef70700801f7800b9d2bf0006
:102880000081fb0002014100214c21004fb1780082
:10289000b9d2bf008080fb0080d2bf000080fb0067
:1028a000008650000c064600204c210060007e008f
:1028b0000ef807000001be00d0948000e194800073
:1028c00032f70700c5f70700c0938800b9d2bf00f0
:1028d0000080fb0000004000214c21006080780057
:1028e0004500dd0030628800d2b9ef00d4b9ef00b6
:1028f0001e00070095f2ae00060037000621ef002b
:102900000a21ef000080eb00219c21000900090052
:10291000801878000400370095f2ae0002003700fe
:102920000621ef000a21ef00a5d2bf00a652e30066
:10293000090032000188af0007003700a672ec00e2
:10294000a6d2bf000080fb0061ad210060c078000e
:102950000080fb00201188009432af0014cea80044
:102960009432ae0014cea90032fc3700b5f2ef006d
:1029700099f2a8004e32ef0071928000e48f50006f
:1029800016003e0070928000c200dd00209c2100f5
:10299000008040001000be000001be00b094800026
:1029a000c1948000800f5100818f590009003100cf
:1029b00070928000c200dd00209c21000080400059
:1029c0001000be00b0948800c19488004ed2bf00b1
:1029d000b5f2b7004e32ec00e7ff3900b612a9009d
:1029e00000000600b1f2ef0000000600aff2bf00e9
:1029f0001600320070c0b300af52e30013003e0077
:102a0000a572ec00a5d2bf000080fb00720b200075
:102a100061ad210002f07800a572ec00a5d2bf00e4
:102a20000081fb0061ad2100afd2bf0000f1780052
:102a3000a572ec00a5d2bf000081fb0061ad2100b2
:102a4000b0d2bf0000f17800d1003700b0c0b300b1
:102a5000af52e30013003a00a572ec00a5d2bf000c
:102a60000080fb00720b200061ad210002f07800b5
:102a7000a572ec00a5d2bf000080fb00b2002000d0
:102a800061ad210002f07800a572ec00a5d2bf0074
:102a90000081fb0061ad2100b0d2bf0000f17800e1
:102aa000bb003700afd2bf00d1c0b30080cf100051
:102ab0001600360030c1b300af52e30013003e00f1
:102ac000a572ec00a5d2bf000080fb00720b2000b5
:102ad00061ad210002f07800a572ec00a5d2bf0024
:102ae0000081fb0061ad2100afd2bf0000f1780092
:102af000a572ec00a5d2bf000081fb0061ad2100f2
:102b0000b0d2bf0000f17800a100370000c4b300cc
:102b1000af52e30013003a00a572ec00a5d2bf004b
:102b20000080fb00720b200061ad210002f07800f4
:102b3000a572ec00a5d2bf000080fb0002042000bb
:102b400061ad210002f07800a572ec00a5d2bf00b3
:102b50000081fb0061ad2100b0d2bf0000f1780020
:102b60008b00370010c4b300af52e30019003a00e5
:102b7000b052e200140036007ab2ef00a572ec0009
:102b8000a5d2bf000080fb00720b200061ad2100c8
:102b900002f07800a572ec00a5d2bf000080fb0017
:102ba000b207200061ad210002f07800a572ec00b0
:102bb000a5d2bf000080fb000200200061ad210013
:102bc00002f07800010037007a32ef007c32ef002b
:102bd0006f00370020c4b300af52e30016003a0084
:102be000a572ec00a5d2bf000080fb00720b200094
:102bf00061ad210002f07800a572ec00a5d2bf0003
:102c00000080fb002204200061ad210002f078006a
:102c1000a572ec00a5d2bf000081fb0061ad2100d0
:102c2000b0d2bf0000f17800b052e20001003a00db
:102c3000590007005600370060c4b300af52e300ec
:102c40000a003a00b0d2bf000080fb000000400044
:102c5000209288004452ec0080f2b700209280005d
:102c60001040b00080f2b7004900370070c4b300d4
:102c7000af52e3000a003a00b0d2bf000080fb0070
:102c800000004000209288004452ec0082f2b7001d
:102c9000209280001040b00082f2b7003c00370064
:102ca00090c4b300af52e3000b003a00f0c7b3008a
:102cb000b052b50005003100b0d2bf000080fb006b
:102cc0004500dd003061880002003700f0ff200081
:102cd000306188002e003700a0c4b300af52e3007b
:102ce00003003a00b0d2bf0086f2b70028003700d8
:102cf000d0c4b300af52e30010003a00b0d2bf001e
:102d000080407800f007200001405000b0f2b7008a
:102d1000f2002000b0d2bf000080fb000200e00003
:102d200002003200110009000280d80020928800c1
:102d30004412ec004094880015003700b0c7b3007f
:102d4000af52e30012003a00a572ec00a5d2bf001a
:102d50000080fb00720b200061ad210002f07800c2
:102d6000a572ec00a5d2bf000080fb00b2072000d6
:102d700061ad210002f07800a572ec00a5d2bf0081
:102d80000081fb0061ad2100b0d2bf0000f17800ee
:102d9000aff2ef0000000600b612a8004e32ef00be
:102da00071928000e48f500009003e007092800014
:102db000c200dd00209c210000814000f0ff2f00b8
:102dc000f1ff2f000089be004e32ec00f4ff390005
:102dd0002368a9007c32ef007ab2ef000000060001
:102de0007cb2ef0000000600c2b8ef00a0c72500cb
:102df00020c688005098250030c6880040812500f4
:102e000040c68800906a250050c6880030542500ce
:102e100060c68800303e250070c6880090282500d6
:102e200080c688005013250090c6880060fe2400ec
:102e3000a0c68800c0e92400b0c6880080d5240060
:102e4000c0c6880090c12400d0c68800f0ad240020
:102e5000e0c68800a09a2400f0c68800a08724005d
:102e600000c78800f074240010c788009062240016
:102e700020c788008050240030c78800b03e24005e
:102e800040c78800302d240050c78800f01b240064
:102e900060c78800000b240070c7880050fa230028
:102ea00080c78800e0e9230090c78800c0d92300cc
:102eb000a0c78800e0c92300b0c7880040ba23003b
:102ec000c0c78800e0aa2300d0c78800c09b2300a9
:102ed000e0c78800e08c2300f0c78800307e230024
:102ee00000c88800d06f230010c88800a0612300ac
:102ef00020c88800b053230030c88800f045230064
:102f000040c888007038230050c88800202b230058
:102f100060c88800101e230070c88800401123007c
:102f200080c888009004230090c8880020f8220000
:102f3000a0c88800e0eb2200b0c88800d0df2200e3
:102f4000c0c88800f0d32200d0c8880050c8220032
:102f5000e0c88800d0bc2200f0c8880080b1220000
:102f600000c9880070a6220010c98800809b22003a
:102f700020c98800c090220030c988002086220025
:102f800040c98800c07b220050c98800807122009f
:102f900060c988006067220070c98800805d2200d7
:102fa00080c98800c053220090c98800204a2200ae
:102fb000a0c98800b0402200b0c988006037220054
:102fc000c0c98800402e2200d0c9880040252200b8
:102fd000e0c98800601c2200f0c98800b0132200fc
:102fe00000ca8800200b220010ca8800b00222000c
:102ff00020ca880060fa210030ca880040f221000f
:1030000040ca880030ea210050ca880050e22100fe
:1030100060ca880090da210070ca8800e0d22100de
:1030200080ca880060cb210090ca8800f0c32100cc
:10303000a0ca8800b0bc2100b0ca880080b52100b9
:10304000c0ca880080ae2100d0ca880090a72100a5
:10305000e0ca8800b0a02100f0ca8800009a2100d0
:1030600000cb88006093210010cb8800e08c210009
:1030700020cb88008086210030cb88003080210062
:1030800040cb8800007a210050cb8800f0732100eb
:1030900060cb8800f06d210070cb880000682100b3
:1030a00080cb88004062210090cb8800805c2100aa
:1030b000a0cb8800e0562100b0cb880060512100f1
:1030c000c0cb8800f04b2100d0cb88009046210077
:1030d000e0cb880050412100f0cb8800203c21004b
:1030e00000cc88001037210010cc8800103221005d
:1030f00020cc8800202d210030cc880040282100e1
:1031000040cc88008023210050cc8800d01e2100b4
:1031100060cc8800301a210070cc8800a0152100f6
:1031200080cc88002011210090cc8800c00c2100a8
:10313000a0cc880070082100b0cc880020042100b9
:10314000c0cc8800f0ff2000d0cc8800d0fb20004d
:10315000e0cc8800c0f72000f0cc8800d0f320003d
:1031600000cd8800e0ef200010cd880000ec2000aa
:1031700020cd880030e8200030cd880070e42000a9
:1031800040cd8800c0e0200050cd880020dd200028
:1031900060cd880090d9200070cd880010d6200026
:1031a00080cd8800a0d2200090cd880040cf2000a4
:1031b000a0cd8800e0cb2000b0cd8800a0c82000c2
:1031c000c0cd880060c52000d0cd880030c220006e
:1031d000e0cd880010bf2000f0cd880000bc2000aa
:1031e00000ce88000000060010c3b300d6fbb70075
:1031f00030c3b300d7fbb70050c3b300d8fbb70050
:1032000070c3b300d9fbb70090c3b300dafbb700bb
:10321000b0c3b300dbfbb700d0c3b300dcfbb70027
:10322000f0c3b300ddfbb70010c4b300defbb70092
:1032300030c4b300dffbb70050c4b300e0fbb700fd
:1032400070c4b300e1fbb70090c4b300e2fbb70069
:10325000b0c4b300e3fbb700d0c4b300e4fbb700d5
:1032600070c3b300e6fbb70090c3b300e7fbb70041
:10327000b0c3b300e8fbb700d0c3b300e9fbb700ad
:10328000f0c3b300eafbb70010c4b300ebfbb70018
:1032900030c4b300ecfbb70050c4b300edfbb70083
:1032a00070c4b300eefbb70090c4b300effbb700ef
:1032b000b0c4b300f0fbb700d0c4b300f1fbb7005b
:1032c000f0c4b300f2fbb70010c5b300f3fbb700c6
:1032d00030c5b300f4fbb70050c5b300f5fbb70031
:1032e00070c5b300f6fbb70090c5b300f7fbb7009d
:1032f000b0c5b300f8fbb700d0c5b300f9fbb70009
:10330000f0c5b300fafbb70010c6b300fbfbb70073
:0833100000000600ffff37007a
:020000040000fa
:10331800401200000e000000800000004e12000065
:10332800440000008000000092120000100000001d
:1033380080000000a21200002000000080000000b1
:10334800c21200000007000080000000c21900003f
:103358001400000080000000d619000026020000ba
:083368008000000000000000dd
:00000001FF
